:100000000C945D000C94360A0C940F0A0C94850035
:100010000C9485000C9485000C94B50A0C94850012
:100020000C9485000C9485000C9485000C9485003C
:100030000C9485000C9485000C9485000C9485002C
:100040000C94C5090C9485000C94830A0C945D0AE9
:100050000C9485000C9485000C9485000C9485000C
:100060000C94A6080C9485000000000024002700D2
:100070002A0000000000250028002B0004040404CE
:100080000404040402020202020203030303030342
:10009000010204081020408001020408102001021F
:1000A00004081020000000080002010000030407FB
:1000B0000000000000000000BF0A11241FBECFEFA7
:1000C000D8E0DEBFCDBF12E0A0E0B1E0E0E0FCE1AF
:1000D00002C005900D92A83EB107D9F724E0A8EE22
:1000E000B2E001C01D92AB3CB207E1F710E0CDE5F4
:1000F000D0E004C02197FE010E94F80DCC35D10755
:10010000C9F70E944D0B0C94FE0D0C940000209139
:100110009F03260F3327331F21323105ECF4209142
:10012000C503FC0190E080E0243069F082E008958E
:10013000A0919F032191AC0143585C4FA40FB52FB0
:10014000B11D2C930196861798F380919F03680F39
:1001500060939F0380E0089581E0089508950895D5
:100160000895E091740380917303E81730F4F0E090
:10017000ED5AFC4F808190E008958FEF9FEF089536
:1001800090917403809173032FEF3FEF981748F419
:10019000E92FF0E0ED5AFC4F208130E09F5F909313
:1001A0007403C90108958091730390917403891BAE
:1001B000990B0895CF92DF92EF92FF920F931F93C6
:1001C000CF93DF937C01CB018A012091520322233C
:1001D00089F0EB016B01C40ED51ECC15DD0569F06D
:1001E0006991D701ED91FC910190F081E02DC7015B
:1001F0000995F3CF642F0E948700C801DF91CF914A
:100200001F910F91FF90EF90DF90CF900895CF93C3
:10021000DF931F92CDB7DEB769832091520322236B
:10022000F9F020917503203258F021E030E0FC0114
:100230003383228390E080E00F90DF91CF91089587
:1002400080917603E82FF0E0EE5CFC4F998190837B
:100250008F5F809376038093750381E090E0ECCF0D
:1002600061E0CE0101960E948700F7CF90E0FC018B
:10027000EC55FF4F2491FC01E057FF4F3491FC01F6
:10028000E458FF4FE491EE23C9F0222339F02330E4
:1002900001F1A8F4213019F1223029F1F0E0EE0F3C
:1002A000FF1FEE58FF4FA591B4918FB7F894EC91D2
:1002B000611126C030953E233C938FBF08952730AF
:1002C000A9F02830C9F0243049F7809180008F7D53
:1002D00003C0809180008F7780938000DFCF84B54A
:1002E0008F7784BDDBCF84B58F7DFBCF8091B0004D
:1002F0008F778093B000D2CF8091B0008F7DF9CFFF
:100300003E2BDACF1092C50381E08093C703109291
:10031000C60361E082E10E94360161E083E10E9450
:100320003601E9EBF0E080818E7F808380818D7FD4
:10033000808388E48093B80085E48093BC000895AE
:10034000CF93DF9391E090937C038823B9F0C09121
:10035000B800D091BA008091BC008A7B8093BC0029
:1003600060E082E10E94360160E083E10E94360194
:100370000E948201D093BA00C093B800DF91CF9160
:1003800008953FB7F89480912E0390912F03A09188
:100390003003B091310326B5A89B05C02F3F19F05B
:1003A0000196A11DB11D3FBFBA2FA92F982F8827F5
:1003B000BC01CD01620F711D811D911D42E0660FD0
:1003C000771F881F991F4A95D1F708958F929F92A2
:1003D000AF92BF92CF92DF92EF92FF924B015C01FE
:1003E0000E94C1016B017C010E94C1016C197D0951
:1003F0008E099F09683E734081059105A8F321E0AD
:10040000821A9108A108B10888EEC80E83E0D81EB0
:10041000E11CF11C81149104A104B10429F7FF909F
:10042000EF90DF90CF90BF90AF909F908F90089506
:100430002FB7F89460912A0370912B0380912C03BD
:1004400090912D032FBF08956091E80281E0682705
:100450006093E8028DE00C943601FC0142835383E3
:100460006483758386819781A085B185840F951FEC
:10047000A61FB71F82879387A487B587089508951D
:10048000AF92BF92CF92DF92EF92FF920F931F93A2
:10049000CF93DF936C017B018B01040F151FEB01E0
:1004A0005E01AE18BF08C017D10759F06991D60197
:1004B000ED91FC910190F081E02DC6010995892B09
:1004C00079F7C501DF91CF911F910F91FF90EF90C8
:1004D000DF90CF90BF90AF900895FC01538D448D75
:1004E000252F30E0842F90E0821B930B541710F0DF
:1004F000CF96089501970895FC01918D828D9817EC
:1005000061F0A28DAE0FBF2FB11D5D968C91928DC3
:100510009F5F9F73928F90E008958FEF9FEF0895F4
:10052000FC01918D828D981731F0828DE80FF11DBD
:10053000858D90E008958FEF9FEF0895FC01918DD8
:10054000228D892F90E0805C9F4F821B91098F73D1
:100550009927089587EF93E00E949E0221E0892B5E
:1005600009F420E0822F089580E090E0892B29F0A3
:100570000E94AA0281110C9400000895FC01A48D30
:10058000A80FB92FB11DA35ABF4F2C91848D90E0B5
:1005900001968F739927848FA689B7892C93A08998
:1005A000B1898C91837080648C93938D848D981322
:1005B00006C00288F389E02D80818F7D80830895B5
:1005C000EF92FF920F931F93CF93DF93EC0181E0A3
:1005D000888F9B8D8C8D98131AC0E889F98980814A
:1005E00085FF15C09FB7F894EE89FF896083E8897D
:1005F000F98980818370806480839FBF81E090E06F
:10060000DF91CF911F910F91FF90EF900895F62EFB
:100610000B8D10E00F5F1F4F0F731127E02E8C8D95
:100620008E110CC00FB607FCFACFE889F9898081DA
:1006300085FFF5CFCE010E94BE02F1CFEB8DEC0F0E
:10064000FD2FF11DE35AFF4FF0829FB7F8940B8FF7
:10065000EA89FB8980818062CFCFCF93DF93EC0161
:10066000888D8823B9F0AA89BB89E889F9898C919A
:1006700085FD03C0808186FD0DC00FB607FCF7CF56
:100680008C9185FFF2CF808185FFEDCFCE010E9456
:10069000BE02E9CFDF91CF9108958F929F92AF92E2
:1006A000BF92CF92DF92EF92FF920F931F93CF935F
:1006B000DF9380911D03882301F1C0901903D0902E
:1006C0001A03E0901B03F0901C03C0921503D09214
:1006D0001603E0921703F09218030E94C101609381
:1006E000190370931A0380931B0390931C032091AA
:1006F0001003222379F010921003DF91CF911F9104
:100700000F91FF90EF90DF90CF90BF90AF909F90B0
:100710008F90089520911E0330911F0337FD13C061
:100720006C197D098E099F0900910E0310910F032A
:1007300030E020E0601771078207930720F481E022
:1007400080931003DACF80911103909112039601E8
:10075000281B390BC0921103D0921203E0921303AD
:10076000F092140380911E0390911F03019609F0EB
:100770004BC0C901815C9241873D974208F0BDCFD3
:1007800010920D03C90168E270E00E94AE0D9B015A
:100790007093020360930103FB01EE0FFF1FE60F4E
:1007A000F71FCF016AE070E00E94AE0D70930F0357
:1007B00060930E03F0930003E093FF02F093FE02B8
:1007C000E093FD0253E0220F331F5A95E1F7309377
:1007D000FC022093FB0280911E0390911F0301965F
:1007E00090931F0380931E0360E08DE0DF91CF9113
:1007F0001F910F91FF90EF90DF90CF90BF90AF903F
:100800009F908F900C94360180911E0390911F034E
:10081000892BD9F48091FF029091000382179307EE
:1008200038F48FEF9FEF90931F0380931E0365CFE3
:1008300010920C0310920A03109203031092040307
:100840001092050310920603C6CF80911E0390916B
:100850001F030197C1F4809101039091020367E0A7
:10086000689FA001699F500D112424173507C8F215
:100870006FE0689FA001699F500D11244217530734
:1008800008F0A9CFCECF80911E0390911F03843929
:1008900091050CF0A0CF9091FA02990F9093FA0273
:1008A0004091FF025091000342175307F0F19E70F0
:1008B0009093FA0280911E0390911F0364E070E010
:1008C0000E94C20D9C01019709F085CF80911E0303
:1008D00090911F038A3691050CF0DBC080910303D1
:1008E00090910403A0910503B0910603880F991F0E
:1008F000AA1FBB1F8093030390930403A0930503D7
:10090000B09306032091FA022F70213009F463CFCF
:10091000243009F086CF8160809303039093040311
:10092000A0930503B093060356CF4091FD0250916A
:10093000FE022417350748F04091FB025091FC025B
:100940004217530710F09160B3CFC0910103D091CB
:10095000020384E18C9FA0018D9F500D1124241768
:10096000350708F45ECF80E58C9FA0018D9F500D68
:1009700011244217530708F454CF91FD52CF8091B0
:100980001E0390911F038339910541F080911E034E
:1009900090911F038338910509F043CF80911E0386
:1009A00090911F038339910519F481E080930B0323
:1009B0004091030350910403609105037091060375
:1009C0008091F0029091F102A091F202B091F302B5
:1009D000481759076A077B0719F590910A03809118
:1009E000F70298131DC090910B038091F8029813A1
:1009F00017C090910C038091F902981311C0909147
:100A000007038091F40298130BC0209108033091E2
:100A100009038091F5029091F6022817390759F0E1
:100A200010920D038CE0E1E0F3E0AEEEB2E0019055
:100A30000D928A95E1F790910D039F5F90930D03BE
:100A400080912203981700F18091ED028111E9CE87
:100A500081E08093ED028090080390900903B12C0F
:100A6000A12CC0900A03D12CF12CE12C009107039A
:100A700010E030E020E0E0912003F0912103CE016E
:100A800009951092ED02CDCE10921F0310921E0315
:100A900034CE80911E0390911F038E3691057CF415
:100AA0008091FA028F70813039F0843009F0B9CE2C
:100AB00081E0809307038FCE109207038CCE809144
:100AC0001E0390911F0382379105D4F49091FA028E
:100AD0009F70913049F068F0943009F0A2CE3093C5
:100AE00009032093080377CE10920903109208039C
:100AF00072CE82E090E090930903809308036BCE5E
:100B000080911E0390911F038238910594F4809187
:100B10000A03880F80930A039091FA029F70913024
:100B200009F459CE943009F07CCE816080930A0399
:100B300052CE80911E0390911F03823991050CF0D3
:100B40004ACE80910C03880F80930C039091FA0297
:100B50009F70913009F43FCE943009F062CE8160ED
:100B600080930C0338CECF92DF92EF92FF920F93D7
:100B70001F93CF93DF93FC01C48121E020935203A4
:100B8000C093EC0210927603109275038485682B53
:100B90008BEE93E00E940701D0917503D13208F0EB
:100BA00092C00E94C1016B017C018091C50381113B
:100BB00065C082E08093C50381E08093C7038FEF17
:100BC0008093C4031092E903D093E803A2E3B3E057
:100BD000E8ECF3E080E0D81385C01092EA0380913E
:100BE000EA03CC0FC82BC093EA038091C60381307F
:100BF00009F07CC01092C6030E94C1016B017C0108
:100C00008091EA038093BB008091780390917903EF
:100C1000A0917A03B0917B03892B8A2B8B2B99F0BF
:100C20000E94C101009178031091790320917A0309
:100C300030917B036C197D098E099F0906171707F0
:100C400028073907E0F18091BC0083FDD9CF85ECFE
:100C50008093BC000E94C1016B017C018091C5039F
:100C6000823009F445C08091C4038F3F61F18091C7
:100C7000C403803241F18091C40325C08091780380
:100C800090917903A0917A03B0917B03892B8A2BF1
:100C90008B2B09F48ACF0E94C10100917803109137
:100CA000790320917A0330917B036C197D098E09B9
:100CB0009F09061717072807390708F076CF809194
:100CC00077030E94A0011092760310927503109290
:100CD0005203DF91CF911F910F91FF90EF90DF9022
:100CE000CF9008959D9191938F5F75CF85EEB0CF92
:100CF0008091780390917903A0917A03B0917B035E
:100D0000892B8A2B8B2B09F4A9CF0E94C10100915A
:100D100078031091790320917A0330917B036C1949
:100D20007D098E099F09061717072807390708F05C
:100D300095CFC5CF089590E080E008950F931F935D
:100D4000CF93DF93EC01EE85FF85309709F009958D
:100D50000E9418026E837F83888799870A811B818E
:100D60002C813D81DC01CB01800F911FA21FB31F9D
:100D70008A879B87AC87BD87DF91CF911F910F91A9
:100D800008950F931F93FC010285138524853585F3
:100D9000401B510B620B730B80E077FF80891F9122
:100DA0000F9108950F931F93CF938C01C62F0E942C
:100DB000B3056C2F6460C8010E94B3056C2F6B7F74
:100DC000C8010E94B30583EC90E00197F1F7CF9141
:100DD0001F910F9108950F931F93CF93DF938C0171
:100DE000D62FC42F607F642B0E94D20680E1D89F4B
:100DF000B00111246C2BC801DF91CF911F910F918D
:100E00000C94D206CF93DF93CDB7DEB728970FB6F9
:100E1000F894DEBF0FBECDBF98E0E4E0F1E0DE0164
:100E2000119601900D929A95E1F79091C20498174E
:100E300008F48FEF90E0880F991F21E030E02C0F2D
:100E40003D1F820F931FFC016081606840E08AEBC8
:100E500094E028960FB6F894DEBF0FBECDBFDF91A9
:100E6000CF910C94EB0641E00E94EB0681E090E00C
:100E7000089585ED8093BC0080917803909179036B
:100E8000A0917A03B0917B030796A11DB11D23E0C9
:100E9000B695A795979587952A95D1F72091BC008F
:100EA00024FD03C01092C50308954091780350912A
:100EB000790360917A0370917B03452B462B472B76
:100EC00069F30097A105B10541F025E32A95F1F7F3
:100ED00000000197A109B109E1CF809177030C943B
:100EE000A001FB0101900020E9F73197AF01461BFB
:100EF000570BDC01ED91FC910280F381E02D099408
:100F00008F929F92AF92BF920F931F93CF93DF93D5
:100F1000CDB7DEB7A1970FB6F894DEBF0FBECDBF39
:100F200019A2423008F44AE08E010F5D1F4F842E53
:100F3000912CB12CA12CA50194010E94D60DE62F75
:100F4000B901CA01EA3004F5E05DD801EE938D01E4
:100F5000232B242B252B79F790E080E0109729F0A4
:100F6000BD0187EF93E00E947107A1960FB6F89438
:100F7000DEBF0FBECDBFDF91CF911F910F91BF900C
:100F8000AF909F908F900895E95CDFCFCF93DF9370
:100F90004AE00E948007EC0166E471E087EF93E08D
:100FA0000E9471078C0F9D1FDF91CF910895CF9301
:100FB000DF93BC0187EF93E00E947107EC0166E4C8
:100FC00071E087EF93E00E9471078C0F9D1FDF9106
:100FD000CF9108950C9471078091E90291E08927DF
:100FE0008093E90280E00E94020769E471E08AEBE5
:100FF00094E00E94EA0781E00E94020765E571E043
:101000008AEB94E00E94EA078091E902882341F08C
:1010100088E08093C60460E08AEB94E00C94B3050A
:101020001092C604F8CF2F923F924F925F926F9228
:101030007F928F929F92AF92BF92CF92DF92EF9268
:10104000FF920F931F93CF93DF9300D000D0CDB7C3
:10105000DEB71C012A013B0109831A832B833C83E1
:1010600065E671E087EF93E00E94EA076091EA028B
:101070007091EB0290E080E04AE00E94800766E415
:1010800071E087EF93E00E9471076FE671E087EFF0
:1010900093E00E94EA074AE0C301B2010E94800780
:1010A00066E771E087EF93E00E94EA07B10190E004
:1010B00080E04AE00E94800766E471E087EF93E0F9
:1010C0000E94710760E871E087EF93E00E94EA07F1
:1010D000C701B6010E94C60768E871E087EF93E098
:1010E0000E94EA0769817A818B819C810E94C607F0
:1010F00064E971E087EF93E00E94EA07C501B4015B
:101100000E94C60782EA91E00E94D7078091EA0216
:101110009091EB0201969093EB028093EA020F907C
:101120000F900F900F90DF91CF911F910F91FF9033
:10113000EF90DF90CF90BF90AF909F908F907F9077
:101140006F905F904F903F902F9008951F920F9255
:101150000FB60F9211242F933F934F935F936F938A
:101160007F938F939F93AF93BF93EF93FF93809160
:10117000B900887F803609F44AC0F0F5883209F456
:10118000A7C018F5803109F49BC0B8F4882309F48E
:10119000F9C0883009F494C0FF91EF91BF91AF91ED
:1011A0009F918F917F916F915F914F913F912F917F
:1011B0000F900FBE0F901F901895883109F488C0CA
:1011C000803251F78093C40314C0803409F49DC069
:1011D00040F48033B9F38833F9F68093C40385EC87
:1011E000B0C0803509F485C0883509F496C08834CC
:1011F00099F60E943907D0CF883909F48CC038F5A8
:10120000883729F050F4883611F0803729F683E0CA
:101210008093C5031092C30357C0883809F47BC07C
:10122000803919F0803809F0B7CF8091C30380323C
:1012300008F071C0E091C30381E08E0F8093C30377
:101240008091BB00F0E0ED55FC4F80833DC0803BBA
:1012500039F0E0F4803A09F479C0883A09F09CCF7B
:1012600084E08093C5031092A00310929F03E09145
:101270009D03F0919E03099580919F0381110FC0FA
:1012800081E080939F0310927D0309C0803C09F4A4
:10129000A6CF883C09F4A3CF883B09F07DCFE0912D
:1012A000A00381E08E0F8093A003F0E0E358FC4F91
:1012B00080818093BB009091A00380919F0329C0FF
:1012C0008091EA038093BB0085EC8093BC0064CFDF
:1012D0009091E9038091E803981758F5E091E903AC
:1012E00081E08E0F8093E903F0E0E853FC4F8081AA
:1012F000E9CFE091E90381E08E0F8093E9038091CB
:10130000BB00F0E0E853FC4F80839091E9038091AB
:10131000E8039817C8F285E8D8CFE091E90381E0A7
:101320008E0F8093E9038091BB00F0E0E853FC4FFF
:1013300080838091C70381115CCF81E08093C603D5
:1013400084EA8093BC001092C50326CF85EC80937D
:10135000BC001092C5038091C303803230F4E09149
:10136000C303F0E0ED55FC4F10826091C30370E0C1
:10137000E091A103F091A20383EA93E00995109212
:10138000C3030ACF1092C40334CF1F920F920FB63B
:101390000F9211242F933F938F939F93AF93BF93FB
:1013A00080912A0390912B03A0912C03B0912D03DF
:1013B0003091290323E0230F2D3758F50196A11D05
:1013C000B11D2093290380932A0390932B03A093AC
:1013D0002C03B0932D0380912E0390912F03A091A5
:1013E0003003B09131030196A11DB11D80932E03EE
:1013F00090932F03A0933003B0933103BF91AF912B
:101400009F918F913F912F910F900FBE0F901F9042
:10141000189526E8230F0296A11DB11DD2CF1F9269
:101420000F920FB60F9211242F933F934F935F9318
:101430006F937F938F939F93AF93BF93EF93FF939C
:10144000E0910201F09103010995FF91EF91BF91A5
:10145000AF919F918F917F916F915F914F913F914C
:101460002F910F900FBE0F901F9018951F920F9203
:101470000FB60F9211242F933F934F935F936F9367
:101480007F938F939F93AF93BF93EF93FF93E091DD
:101490000001F09101010995FF91EF91BF91AF918A
:1014A0009F918F917F916F915F914F913F912F917C
:1014B0000F900FBE0F901F9018951F920F920FB6AE
:1014C0000F9211242F933F934F935F936F937F93CA
:1014D0008F939F93AF93BF93EF93FF9387EF93E027
:1014E0000E94BE02FF91EF91BF91AF919F918F91AA
:1014F0007F916F915F914F913F912F910F900FBE10
:101500000F901F9018951F920F920FB60F921124F3
:101510002F938F939F93EF93FF93E0910704F091A4
:1015200008048081E0910D04F0910E0482FD1BC03F
:101530009081809110048F5F8F7320911104821726
:1015400041F0E0911004F0E0E950FC4F958F80935A
:101550001004FF91EF919F918F912F910F900FBEEB
:101560000F901F9018958081F4CF1F920F920FB6A5
:101570000F9211240F900FBE0F901F901895EF92AD
:10158000FF921F93CF93DF93EBEEF3E0138212826F
:1015900088EE93E0A0E0B0E084839583A683B783D0
:1015A00020E131E031832083E7EFF3E01382128200
:1015B00084839583A683B78382E291E091838083BD
:1015C00085EC90E09587848784EC90E09787868708
:1015D00080EC90E0918B808B81EC90E0938B828B00
:1015E00082EC90E0958B848B86EC90E0978B868BD9
:1015F000118E128E138E148EEAEBF4E01382128297
:101600008EE391E091838083118687E2848380E179
:10161000828782E083871486C7EAD4E084E3E82ED9
:1016200081E0F82EF982E88211E0188B1F861E8671
:101630001A861B861C861D860E9418026E837F8375
:1016400088879987DA8BC98B1A821B821C821D823C
:101650006A877B878C879D87C4E9D4E0F982E8821A
:10166000188B1F861E861A861B861C861D860E9466
:1016700018026E837F8388879987DA8BC98B1A82D9
:101680001B821C821D826A877B878C879D87DF91E6
:10169000CF911F91FF90EF900895CF93DF9300D0EB
:1016A000CDB7DEB7789484B5826084BD84B581609F
:1016B00084BD85B5826085BD85B5816085BD80911D
:1016C0006E00816080936E00109281008091810095
:1016D000826080938100809181008160809381008D
:1016E000809180008160809380008091B10084604F
:1016F0008093B1008091B00081608093B0008091B0
:101700007A00846080937A0080917A00826080936E
:101710007A0080917A00816080937A0080917A00CB
:10172000806880937A001092C100E0910704F091E4
:10173000080482E08083E0910304F09104041082A5
:10174000E0910504F091060480E1808310920F047B
:10175000E0910B04F0910C0486E08083E091090491
:10176000F0910A04808180618083E0910904F09106
:101770000A04808188608083E0910904F0910A0462
:10178000808180688083E0910904F0910A0480815F
:101790008F7D808387ED91E00E94D70769E072E03A
:1017A00087EF93E00E94EA078EE292E00E94D7075B
:1017B00067E372E087EF93E00E94EA0784E492E037
:1017C0000E94D707EDE9F0E02491E9E8F0E0849188
:1017D000882399F090E0880F991FFC01E859FF4F8A
:1017E000A591B491FC01EE58FF4F859194918FB76C
:1017F000F894EC91E22BEC938FBFE2E9F0E02491B6
:10180000EEE7F0E084918823C9F090E0880F991FFB
:10181000FC01E859FF4F45915491FC01EE58FF4FF0
:10182000A591B4919FB7F894FA013081822F8095E9
:1018300083238083EC91E22BEC939FBF109274037F
:101840001092730310927603109275030E94820126
:101850008EEA90E090939E0380939D038FEA90E040
:101860009093A2038093A1031092BF048091C504BA
:10187000823018F098E09093BF048093C20462E332
:1018800070E080E090E00E94E6016091C6048AEB7F
:1018900094E00E94B30568EE73E080E090E00E945F
:1018A000E60160E38AEB94E00E94D2060BE416E4C2
:1018B000C8010197F1F760E38AEB94E00E94D20639
:1018C000C8010197F1F760E38AEB94E00E94D20629
:1018D00083E592E00197F1F760E28AEB94E00E94E1
:1018E000D2066091BF04606240E08AEB94E00E94FF
:1018F000EB0684E08093C00440E06CE08AEB94E067
:101900000E94EB0640E061E08AEB94E00E94EB0667
:101910008BE39FE10197F1F78091C304882319F0CD
:1019200080E00E94020712E01093C10440E066E0EC
:101930008AEB94E00E94EB0640E062E08AEB94E0E0
:101940000E94EB068BE39FE10197F1F784E292E0BE
:101950009093B6048093B5044CED55E060E070E0E0
:101960004093A9045093AA046093AB047093AC0411
:101970008091AD049091AE04A091AF04B091B004F9
:1019800084529A4FAF4FBF4F8093B1049093B204EB
:10199000A093B304B093B4048CEE97E09093A304A7
:1019A0008093A20440939604509397046093980404
:1019B0007093990480919A0490919B04A0919C0447
:1019C000B0919D0484529A4FAF4FBF4F80939E04B5
:1019D00090939F04A093A004B093A10410922303BA
:1019E0001093220383E198E09093210380932003D6
:1019F0008FEF9FEF90931F0380931E0381E08093EE
:101A00001D038DE493E09093010180930001809188
:101A100069008C7F816080936900E89A80E592E09C
:101A20000E94D70785E692E00E94D70780E992E0FE
:101A30000E94D70760ED77E080E090E00E94E60129
:101A40008EEA92E00E94D70760ED77E080E090E0B8
:101A50000E94E601CE0101965C0100E010E09924AD
:101A600093940E9418022B013C018091280381115C
:101A70003FC08CEC92E00E94D7076CED72E087EFDC
:101A800093E00E94EA078091C7049091C8040097F0
:101A900011F48BEC94E06501C81AD90A0D2C000CE6
:101AA000EE08FF084AE0C701B601F7FE0DC06DE27F
:101AB00087EF93E00E94E00266277727CB016C193D
:101AC0007D098E099F094AE00E94800766E471E063
:101AD00087EF93E00E94710787ED91E00E94D7079E
:101AE0009092280368EE73E080E090E00E94E601A7
:101AF0000E941802AB01BC0184E994E00E94C10677
:101B0000882321F084E994E00E949E0680912403BA
:101B100090912503A0912603B0912703481A590AF2
:101B20006A0A7B0A98EC491651046104710450F06A
:101B30000E94180260932403709325038093260368
:101B4000909327030115110509F48BCF0E94AA0277
:101B5000882309F486CF0E94000083CFAA1BBB1BF9
:101B600051E107C0AA1FBB1FA617B70710F0A61B9D
:101B7000B70B881F991F5A95A9F780959095BC01BE
:101B8000CD01089597FB072E16F4009407D077FD3A
:101B900009D00E94AE0D07FC05D03EF490958195CA
:101BA0009F4F0895709561957F4F0895A1E21A2E79
:101BB000AA1BBB1BFD010DC0AA1FBB1FEE1FFF1FF1
:101BC000A217B307E407F50720F0A21BB30BE40B41
:101BD000F50B661F771F881F991F1A9469F7609588
:101BE0007095809590959B01AC01BD01CF01089542
:101BF000EE0FFF1F0590F491E02D0994F894FFCFAC
:101C00003F023F02000040001400540000000000AA
:101C10000701DA009B06B000D300C000B10000004D
:101C20000000E00240026D022D039E027C02900241
:101C3000000000002D02C1069E06000000003307D0
:101C400040029B069A060D0A00415A2D44656C69B4
:101C50007665727900456E6A6F79202D2041726435
:101C600075696E6F00436F756E7465723A2000433C
:101C70006F64653A200020506572696F643A2000F5
:101C800020756E69743A20002067726F7570426922
:101C9000743A200020737769746368547970653AE8
:101CA00020002D2D2D2D2D2D2D2D2D2D2D2D2D2D9E
:101CB0002D2D2D2D2D2D2D2D2D2D2D2D2D2D2D2D54
:101CC0002D2D2D2D2D2D2D2D2D2D2D2D2D2D2D2D44
:101CD0002D2D2D2D2D2D002A2A2A2A2A2A2A2A2A7C
:101CE0002A2A2A2A2A2A2A2A2A2A2A2A2A2A2A2A54
:101CF0002A2A2A2A2A2A2A2A2A2A2A2A2A2A2A2A44
:101D00002A2A2A2A2A2A2A2A00426F617264206912
:101D10006E697469616C697A656420737563636563
:101D2000737366756C6C793A20007372632F6D6102
:101D3000696E2E637070004275696C642064617412
:101D4000653A20004D61722020342032303231005B
:101D5000526563656976657220696E697469616C44
:101D6000697A6564003134434F5245207C205246E5
:101D700020536E6966666572205465737420436FE4
:101D8000646520666F7220526563656976657200CE
:101D9000524620536E696666657220496E697469A1
:101DA000616C697A696E672E2E2E2E2E2E0053746A
:101DB000617274696E672E2E2E2E2E2E2E2E2E2ED2
:101DC0002E2E2E2E2E2E2E2E2E2E2E00456E74658D
:101DD00072696E67206C6F6F7028290046726565A6
:081DE0002052414D3A200000A1
:00000001FF
